:02000000F628E0
:02000800D628F8
:04000C000D08820752
:1000100007340F340034FF340D08820707340F34DF
:100020000234FF340D08820707340F340434FF34E0
:100030000D08820707340F340834FF340D08820797
:1000400007340F341034FF340D08820707340F349F
:100050002034FF340D08820707340F340534FF3491
:100060000D08820707340F340934FF340D08890066
:10007000831608148312080808000D088207093443
:1000800002340034FF34A01B002AC8309500093028
:100090006C2000308D0085194B280D08890006085A
:1000A00088008E008316081555308900AA30890013
:1000B000881408118312851D5B280608FF3A03196E
:1000C000642897208D0A4B2803308E009000FF3063
:1000D00095009720A0176B288C008D0103100C0D44
:1000E0008207062085280C208528122085281820C4
:1000F00085281E208528242085282A208528302030
:100100008528362085283D2085288E008E080319F5
:100110009328FF300E060319080097208D0A02303D
:100120008F00C3206E2804308F00C3208E28031058
:100130008E0C8E0803190800031C9F28A728013085
:1001400090008F008514B0208510C32097280330BD
:10015000900001308F008514B0208510C3209728AF
:1001600010089100150892000514B2309300930B0B
:10017000B7280510B2309300930BBC28920BB4281B
:10018000910BB22808000F08910015089200141472
:10019000B2309300930BCA281410B2309300930B23
:1001A000CF28920BC728910BC52808009600030E94
:1001B0009700980BF02810309800990BF0283C30ED
:1001C0009900A60BE8280A30A6009E030319201404
:1001D0009C0AA0141C081D02031DF02801309C007D
:1001E0000B11170E8300960E160E090007306200E1
:1001F0008501860118306500FF30660085194328A7
:0602000001308A000A290A
:0C021400810164008B018B178B161030E9
:1002200098003C3099000A30A600A00120219E08C9
:10023000031D682118309E0073218B13630000009A
:100240000608073925219E002E2982070034033431
:10025000063409340C340F34123415340608383996
:100260009A0003109A0C9A0C9A0C1A083C219F00D1
:100270001A084521A2004E298207003401340234B5
:10028000033404340534063407348207013401345E
:100290000234033404340534063407349A01061F4B
:1002A00052291A14861F55299A14051E58291A1501
:1002B0001A084521013E9D001D08220203186121F4
:1002C000080018080239031D8514031985106129D7
:1002D000201018080F3903198514031D8510201CE0
:1002E00069298510080001309C00A00120111C081C
:1002F0002206031D20152018080020197629A010B9
:1003000005159130950000308A001F086C201908EF
:10031000363A031D87291F086C201908303A031D3F
:100320008D291F086C2019082A3A031D93291F08DC
:100330006C201908243A031D99291F086C201908FC
:100340001E3A031D9F291F086C201908183A031D27
:10035000A5291F086C201908123A031DAB291F0894
:100360006C2019080C3A031DB1291F086C201908CC
:10037000063A031DB7292D30950009306C2008304E
:0E0380006C2001308A00A01CC32905117629CB
:100400008514052285100522002AFF30A300A400D0
:0E041000A30B082AFF309600A40B082A080050
:02400E00F13F80
:0E42000014000F00190011000F001900FF003C
:00000001FF
